:100000000C94D9000C94F6000C94F6000C94F600B5
:100010000C94F6000C94F6000C94F6000C94F60088
:100020000C94F6000C94F6000C94F6000C94F60078
:100030000C94F6000C94F6000C94F6000C94F60068
:100040000C94F6000C94F6000C94F6000C94F60058
:100050000C94F6000C94F6000C94F6000C94F60048
:100060000C94F6000C94F6005A016B0183018C0588
:100070008C05B001B6028C058C058C058C058C05B1
:100080008C058C058C05F30164026802570154014C
:100090009202740416052D0516052D052D052D0556
:1000A0004D0599059B058C058C058C058C058C05EB
:1000B0008C058C058C058C058C058C058C058C05B8
:1000C0008C05A401910194018C0597019901A4016B
:1000D0009B059B018C05A6018C058C0599059E014D
:1000E000A1011B5B306D1B5B324A1B5B303B3066F2
:1000F0000052656164792E204A75737420636C6FB9
:10010000736520746865207465726D696E616C2E0C
:10011000204E6F207265736574206E65656465643A
:100120002E0D0A002028686578290D0A000D0A4F57
:100130004B2C206D792053572076657273696F6E52
:10014000206973206E6F773A20005D3A2000456E7B
:100150007465722053572056657273696F6E204D17
:10016000696E6F7220696E20686578205B005D3A69
:100170002000456E7465722053572056657273696E
:100180006F6E204D616A6F7220696E2068657820FD
:100190005B004176725573623530302D312E3761F8
:1001A000207465726D696E616C206D6F64650D0AF7
:1001B000000011241FBECFEFD4E0DEBFCDBF11E0A1
:1001C000A0E0B1E0E8E3F2E102C005900D92AC30AE
:1001D000B107D9F712E0ACE0B1E001C01D92AF3336
:1001E000B107E1F70E947F060C941A090C940000F5
:1001F000A0E0B0E0EEEFF0E00C948F08082FEB01E8
:100200009B012150304081E02D31380728F080ECEF
:1002100080930D01C2E0D0E08BE10E945607802F51
:100220000E9456076E01ED2C8D2D0E9456078C2FD3
:100230000E9456078EE00E94560785E1B82EB02630
:10024000BC26BD240E9484080CE011E0CC24DD24EF
:100250000CC07801F80181918F010E945607F701C7
:100260008081B8260894C11CD11CCC16DD0688F309
:100270008B2D0E945607CDB7DEB7E9E00C94AB0892
:10028000A0E0B0E0E6E4F1E00C948608282E80912E
:100290000C0190E001978D31910508F03DC48C5C14
:1002A0009F4FFC010C94BD08DD24D3941EC3DD24B4
:1002B000D39439C181E080930C0110920D0188E044
:1002C00080930E018FE091E060E071E00E94C3082E
:1002D0006BE070E026C480910D01883929F480918B
:1002E0000E010E949E071BC18E3929F480910E01D8
:1002F0008093090114C18F3909F011C180910E0159
:10030000809333020CC180910D0190E080589040A1
:100310008032910508F000C48F5A9F4FFC010C9465
:10032000BD0880913D0214C080913E0211C082E35D
:1003300012C089E110C00E94D5070AC0809109014E
:1003400007C08091330204C082E005C08CE803C07E
:100350008F3F09F4E1C310920D0180930E017AC31F
:1003600070910D0160910E01872F90E0A0E0B0E048
:10037000B82FAA2799278827262F30E040E050E0A1
:10038000A90133272227822B932BA42BB52B209155
:10039000100130E040E050E0822B932BA42BB52BD2
:1003A00020910F0130E040E050E0542F432F322FD6
:1003B0002227822B932BA42BB52B8093340290936E
:1003C0003502A0933602B093370277FF04C081E074
:1003D0008093380202C0109238026093390281E0A3
:1003E00080933A029CC0459A0E94F80780910E01C2
:1003F00090E00E946D0880EC80930D0180911001C7
:10040000813318F080E380931001809111018823DB
:1004100019F481E080931101C0E0D0E04DC00E944A
:100420008408459A80910F0190E00E946D088091A8
:1004300014010E9414088091110190E00E946D083F
:10044000809115010E9414088091110190E00E9492
:100450006D084598809116010E941408182F80910C
:10046000110190E00E946D08809117010E9414080C
:1004700090911301933029F480911201181759F4C7
:1004800008C020911201821711F410920D019923D6
:1004900011F410920D0180910D01882331F4459AD9
:1004A00080911001C82FD0E007C021960E94D80784
:1004B00084E190E00E946D088091100190E0C817DF
:1004C000D90708F4ACCF2BC30E946408459827C015
:1004D00080910F010E941408809110010E9414085D
:1004E000809111010E941408809112010E94140849
:1004F00080910E01882311F006E907C080910D015B
:1005000090E00E946D080BC0015060E070E080E058
:1005100090EF0E94490880FF02C00023A9F71092C3
:100520000D01FDC2DD2480911001843018F484E0B7
:100530008093100180911001813218F080E2809345
:100540001001809134029091350290933C02809387
:100550003B0290910D0180E060900E017724682AA3
:10056000792AF9E16F16F1E07F0610F080ECD5C230
:100570000E948408B0900F01B0FE0AC006E1A02ED0
:1005800001E0B02EC0E0D0E0EE24FF24870141C19D
:1005900016E1812E11E0912EC0E0D0E0EE24FF2480
:1005A0008701AA24B6E9CB2EA2E03A2E96C0DD2020
:1005B00031F0C0FF04C080911101886002C08091B9
:1005C00011010E94140880913402909135020E941A
:1005D0003F082401D4018D914D010E94140890918F
:1005E0001401F2018081981799F0E0903402F090A4
:1005F000350200913602109137028FEF9FEFA0E095
:10060000B0E0E822F9220A231B23B0920F0102C0B6
:1006100030920F010E948408DD2021F482E090E0F6
:100620000E946D0880910F0182FF25C08091140106
:10063000F6E9CF2EE1E04E2E512C4C225D2214C063
:10064000DD2039F04114510421F0809113018860BC
:1006500002C0809113010E941408C7010E943F0844
:1006600080E00E941408CA94909114018917C9F47B
:10067000CC2031F716C083FF0FC076E9C72E01C02A
:10068000CA9460E070E080E090EF0E94490880FF2B
:1006900008C0CC20A9F705C08091100190E00E940D
:1006A0006D08DD2011F0C0FF13C0809134029091DD
:1006B0003502A0913602B09137020196A11DB11DFD
:1006C0008093340290933502A0933602B0933702A0
:1006D000CC2011F460E8A62E2196C615D70508F4A3
:1006E00066CFFFC00E94840880913802882309F1F8
:1006F0008091340290913502A0913602B091370278
:10070000A070B0700097A105B10521F080913A0268
:10071000882379F08DE40E94140880E00E94140878
:10072000809139020E94140880E00E9414081092FF
:100730003A02DD2031F0C0FF04C0809111018860D1
:1007400002C0809111010E9414088091340290919E
:1007500035020E943F084501D5018D915D010E943F
:10076000140890911401F4018081981789F0E090A9
:100770003402F090350200913602109137028FEF6B
:100780009FEFA0E0B0E0E822F9220A231B2306C075
:1007900080910F018078806180930F01DD2029F125
:1007A000C0FF36C08091340290913502A09136028C
:1007B000B09137020196A11DB11D80933402909330
:1007C0003502A0933602B0933702A070B0708F3F0D
:1007D000EFEF9E07E0E0AE07E0E0BE07C9F48091CE
:1007E00039028F5F8093390213C080913402909157
:1007F0003502A0913602B09137020196A11DB11DBC
:100800008093340290933502A0933602B09337025E
:100810002196C615D70508F465CF0E9484088091FB
:100820000F0187FF57C0809112010E941408809128
:100830003B0290913C020E943F0880E00E94140815
:10084000DD2021F481E090E00E946D0880910F018D
:1008500085FF28C0E114F1040105110519F180910B
:10086000140156E9D52EE701C170D07011C0209750
:1008700021F080911301886002C0809113010E94D1
:100880001408C7010E943F0880E00E941408DA940F
:1008900090911401891719F4DD2049F71DC0DD205E
:1008A000D9F018C086FF11C006E901C0015060E010
:1008B00070E080E090EF0E94490880FF03C00023B1
:1008C000A9F70DC0002359F005C08091100190E0F8
:1008D0000E946D08AA2405C040E8A42E02C031E899
:1008E000A32EA0920D011BC1DD2490910D0180E08B
:1008F00020910E01C22FD0E0C0900F01C82BD92B40
:10090000F1E0C931DF0710F0C8E1D1E02EE0E22EBE
:1009100021E0F22E00E010E098E0B92EBC2879C06A
:100920000E94840880913802882309F18091340262
:1009300090913502A0913602B0913702A070B0704C
:100940000097A105B10521F080913A02882379F042
:100950008DE40E94140880E00E94140880913902FE
:100960000E94140880E00E94140810923A02DD20D0
:1009700021F000FF02C08B2D01C08C2D0E941408B5
:1009800080913402909135020E943F0880E00E94DD
:100990001408D7018D937D01DD2031F100FF37C0B0
:1009A0002091340230913502409136025091370245
:1009B0002F5F3F4F4F4F5F4F2093340230933502EC
:1009C0004093360250933702407050702F3FBFEF74
:1009D0003B07B0E04B07B0E05B07C9F480913902F8
:1009E0008F5F8093390213C0809134029091350259
:1009F000A0913602B09137020196A11DB11D8093DE
:100A0000340290933502A0933602B09337020F5F01
:100A10001F4F0C171D0708F483CFBE016D5F7F4F7A
:100A200010920D01C45FDE4F1A827BC080910D01D0
:100A30000E94140880910E010E94140880910F01F9
:100A40000E941408809110010E94140810920D0158
:100A500010920E0163E070E064C00EE011E0C0E0AF
:100A6000D0E02196F80181918F010E941408209115
:100A70000D0130E02C173D0711F480930E0185E045
:100A800090E00E946D08C430D10559F710920D0115
:100A900010920F0164E070E044C0E0900E01D0902D
:100AA0000F0110E000E01EC085E090E00E946D089C
:100AB0001D1580F00E1570F4E12FF0E0E45FFE4F9D
:100AC00084810E941408E02FF0E0E45FFE4F8283EF
:100AD0000F5F07C0E12FF0E0E45FFE4F84810E94CA
:100AE00014081F5F80910D011817F0F207C0845F92
:100AF0009E4FDC0112961C9212970F5F802F90E0A0
:100B00000E15A8F3BC016D5F7F4F10920D01845F3D
:100B10009E4FFC01128205C089EC80930D0162E0BA
:100B200070E0822D0E94F800CDB7DEB7E2E10C94B0
:100B3000A20880E010CC81E00ECCA1E0B0E0E3EAB6
:100B4000F5E00C949208882319F4FF24F39402C072
:100B500042E0F42E81E00E947F07082F1FEF32E071
:100B6000E32E2BC0902F90539A3038F0802F815471
:100B7000863018F080528630E0F41F3F09F410E010
:100B8000802F99830E94560799819A3020F41295FC
:100B9000107F190F0DC0902F9154812F8295807F67
:100BA000963018F4102F175302C0102F1755180F36
:100BB000EA9481E00E947F07082F0D3041F00A304F
:100BC00031F0EE2079F604C081E00E947F07FA94AC
:100BD000FF20D1F7812F2196E6E00C94AE088BE13F
:100BE0000E94560785E40E94560708951F93182F08
:100BF00082EE90E00E94710782E991E00E94710705
:100C000082E791E00E94710780913D0290E06CE0E4
:100C100071E040E150E00E94CA088CE091E00E943F
:100C20005D078EE691E00E947107812F0E949D056D
:100C30008F3F11F080933D020E94EF058EE491E01A
:100C40000E94710780913E0290E06CE071E040E10B
:100C500050E00E94CA088CE091E00E945D078AE49F
:100C600091E00E947107812F0E949D058F3F11F036
:100C700080933E020E94EF0581E090E060913E0289
:100C80000E94E80882E090E060913D020E94E8083E
:100C900080E090E064E10E94E8088DE291E00E942B
:100CA000710780913D0290E06CE071E040E150E01E
:100CB0000E94CA088CE091E00E945D078EE20E94CB
:100CC000560780913E02803118F480E30E94560757
:100CD00080913E0290E06CE071E040E150E00E94C3
:100CE000CA088CE091E00E945D0784E291E00E94D6
:100CF000710781EF90E00E9471071F910895A4E0B1
:100D0000B0E0E5E8F6E00C948F088AE090E00E94FD
:100D10004B070E9478083D9A4598789484E0809328
:100D20003E0282E080933D0280E090E00E94E00875
:100D3000843161F481E090E00E94E00880933E02FB
:100D400082E090E00E94E00880933D0260E070E065
:100D500000E010E0BB24FF2440E0F0EBDF2EE1ECEC
:100D6000EE2E0CC05BE1C52E91E015C096E013C0DD
:100D700060E070E000E010E0BB2440E081E04A83E6
:100D80006B837C830E947F07282F4A816B817C8143
:100D90008B3181F4E7CF80E04A836B837C83998336
:100DA0000E947F07282F99814A816B817C81913035
:100DB00021F51FC08D3011F08A30D1F66F5F7F4F63
:100DC000FF2041F42A3009F060C04D3009F05DC0C9
:100DD000FF24F3946430710509F05BC081E001C029
:100DE00080E029830E94F6052981422F60E070E0AF
:100DF000C5CFC826B82E92E0CECF923029F4C826AF
:100E0000182F00E093E0C7CF933031F4C82630E0CC
:100E1000022B132B94E0BFCF943041F4C8268E30C0
:100E200009F0ACCF60E070E095E0B5CF9530B1F45B
:100E3000601771070CF09CCF81E0683178070CF0E7
:100E400097CFC226FB01E45FFE4F20836F5F7F4F89
:100E5000A8956017710709F09ECF88CF963009F0EA
:100E600087CF8C1541F4101611062CF4A8958B2D04
:100E70000E9440017DCFD0920C01E0920D018B2D9C
:100E800062E070E00E94F80073CF6230710509F4EF
:100E9000A7CF422F73CF9093C5008093C40088E101
:100EA0008093C10086E08093C20008959091C000B5
:100EB00095FFFCCF8093C6000895EF92FF92CF93E9
:100EC000DF93E82EE7017E01F92EE70102C00E94C0
:100ED000560789918823D9F7DF91CF91FF90EF9042
:100EE0000895CF93DF93EC0102C00E945607FE01E4
:100EF000219684918823C9F7DF91CF910895A1E0CD
:100F0000B0E0E5E8F7E00C94960806C0882321F0ED
:100F100089830E94840889819091C00097FFF6CF51
:100F20008091C6002196E2E00C94B20802C0809144
:100F3000C6008091C00087FDFACF089510920A0183
:100F4000843028F081E080930A018CE01EC0833059
:100F500031F49DB59E7F9DBD9CB5926012C08230DC
:100F600049F49DB59E7F9DBD9CB592609CBD9CB58E
:100F70009E7F0AC0813061F49DB59E7F9DBD9CB56A
:100F80009D7F9CBD9CB591609CBD80930B01089595
:100F90008DB58E7F8DBD8CB58E7F8CBD8CB58D7FD4
:100FA0008CBD10920B0180E0089580910B01089593
:100FB0008CB51CBC2D98E3EFF1E03197F1F700C040
:100FC00000002D9AE3EFF1E03197F1F700C0000047
:100FD0002D988CBD08952A9A83EF91E00197F1F73F
:100FE00000C000002A9884E190E00E946D080895F6
:100FF000229A2A9A239A2B98259A2D9884E190E098
:101000000E946D0880910A01882331F481E58CBD2E
:1010100080910B010E949E072A9884E190E00E9433
:101020006D080E94EB070895482F80910A018823DC
:1010300031F44EBD0DB407FEFDCF8EB508952D9849
:1010400028E030E080E090E8592F542311F02B9AEB
:1010500001C02B98E3EFF1E03197F1F700C00000F9
:101060001C99892B2D9AE3EFF1E03197F1F700C03D
:1010700000002D9896952150304031F708951F9328
:10108000182F892F0E941408812F0E9414081F9185
:101090000895A2E0B0E0EFE4F8E00C949508182F72
:1010A000892F6A8379830E941408812F0E94140873
:1010B0007981872F0E9414086A81862F0E94140864
:1010C0002296E3E00C94B1081CBC2A9A23982B9832
:1010D00025982D9822982A98089507C0EFEBF2E101
:1010E0003197F1F700C0000001970097B9F7089514
:1010F0002FE088E190E00FB6F894A8958093600007
:101100000FBE209360000895A89508952F923F92F6
:101110004F925F926F927F928F929F92AF92BF9207
:10112000CF92DF92EF92FF920F931F93CF93DF93B3
:10113000CDB7DEB7CA1BDB0B0FB6F894DEBF0FBE10
:10114000CDBF09942A88398848885F846E847D845D
:101150008C849B84AA84B984C884DF80EE80FD805F
:101160000C811B81AA81B981CE0FD11D0FB6F894D5
:10117000DEBF0FBECDBFED010895EE0FFF1F05903E
:10118000F491E02D0994FB01DC0101900D92002007
:10119000E1F70895FB019F01423074F0453264F499
:1011A000642F77270E940609805D8A330CF0895DE1
:1011B0008193CB010097A1F71082C9010C94F60826
:1011C000F999FECF92BD81BDF89A992780B508950F
:1011D000262FF999FECF1FBA92BD81BD20BD0FB653
:1011E000F894FA9AF99A0FBE01960895DC01FC0171
:1011F000672F71917723E1F7329704C07C916D934B
:1012000070836291AE17BF07C8F30895AA1BBB1B7A
:1012100051E107C0AA1FBB1FA617B70710F0A61BF6
:10122000B70B881F991F5A95A9F780959095BC0117
:08123000CD010895F894FFCFF1
:0C1238004156524953505F320001010C36
:00000001FF
